:1000000012C0ADC2E0C22AC089C128C027C026C024
:1000100025C024C023C022C021C020C01FC01EC0D4
:100020001DC01CC01BC011241FBECFE5D4E0DEBF25
:10003000CDBF11E0A0E6B0E0E2EDFDE002C005902A
:100040000D92A236B107D9F711E0A2E6B1E001C0E6
:100050001D92AD36B107E1F73CD3BAC600C01F927E
:100060000F920FB60F9211240F900FBE0F901F909A
:10007000189590E08F70907008952F923F924F9254
:100080005F926F927F928F929F92AF92BF92CF9228
:10009000DF92EF92FF920F931F93CF93DF93CDB731
:1000A000DEB728970FB6F894DEBF0FBECDBF988796
:1000B0008F837A836983842E190110E08E2D90E05E
:1000C000880F991F880F991F081B190B942E8E2DCE
:1000D00090E0A0E0B0E08B839C83AD83BE832801D9
:1000E000662457FC6094762CAFC0AF81B8858C91A4
:1000F0008F608C93F101E90DF11D808190E08F708C
:100100009070E981FA818083F1E09F1671F09F166B
:1001100038F082E0981689F093E09916C9F413C07C
:10012000AF81B8858C918E7F0CC0EF81F88580817E
:100130008D60808380818D7F0AC0AF81B8858C916E
:100140008B7F8C9305C0EF81F8858081877F8083CA
:100150006B817C818D819E81EDD25B016C0120E001
:1001600030E04AE753E440D57B018C0120E030E0E9
:1001700040E85FE3E4D488231CF481E090E020C0F1
:1001800020E03FEF4FE757E4C801B701DCD4181671
:100190009CF420E030E040E251E4C601B50124D5F2
:1001A00065D406C089E190E00197F1F76150704095
:1001B00061157105B9F706C0C801B70157D4CB0165
:1001C0000197F1F7992011F09A943EC0AF81B8855C
:1001D0008C918F608C93C301B20176D45B016C016A
:1001E00020E030E04AE753E4FFD47B018C0120E0BB
:1001F00030E040E85FE3A3D488231CF481E090E082
:1002000020C020E03FEF4FE757E4C801B7019BD47F
:1002100018169CF420E030E040E251E4C601B5013C
:10022000E3D424D406C089E190E00197F1F761504E
:10023000704061157105B9F706C0C801B70116D441
:10024000CB010197F1F7982C80916000882309F089
:100250004CCFEF81F88580818F60808328960FB620
:10026000F894DEBF0FBECDBFDF91CF911F910F91EC
:10027000FF90EF90DF90CF90BF90AF909F908F90C6
:100280007F906F905F904F903F902F9008958FE7F1
:1002900087BB88BB8FE084BB11BA8EE082BB20E1B4
:1002A00037E289E190E00197F1F721503040C9F73A
:1002B0000895FC019B0147E16137740728F0108223
:1002C0001182128213820895CB0168E572E017D57E
:1002D000608370E088E592E0AC01649FC001659F97
:1002E000900D749F900D1124281B390BC9016CE3EC
:1002F00070E005D561838CE3689FB0011124261B53
:10030000370BC9016AE070E0FAD462838AE0689F23
:10031000B0011124261B370B238308951F920F92DF
:100320000FB60F9211242F933F934F935F936F93C8
:100330007F938F939F93AF93BF93EF93FF9380919E
:1003400068018F5F80936801843020F1109268010A
:1003500060916B0170916C016150704070936C0101
:1003600060936B01C49A6115710521F082E691E0FA
:10037000A0DF10C01092620110926301109264011C
:100380001092650185B5887F85BD81E08093690104
:100390001092600080916801823009F4C498FF9146
:1003A000EF91BF91AF919F918F917F916F915F91ED
:1003B0004F913F912F910F900FBE0F901F90189566
:1003C000EF920F938BB780688BBF85B7886085BF2E
:1003D0008BB780648BBF85B7826085BF789481E0DE
:1003E0008093600032E0E32E0EE022E631E043E04D
:1003F00065E370E088E390E040DEF8948BB78F7798
:100400008BBF85B7877F85BF8BB78F7B8BBF85B74A
:100410008D7F85BF0F91EF900895FC01DB018081F6
:1004200090E028E532E0A901849F9001859F300D7E
:10043000949F300D11248381280F311D81814CE35D
:10044000849FC0011124280F391F82814AE0849FB4
:10045000C0011124280F391F2D933C930895EF926A
:100460000F938BB780648BBF85B7826085BF89B7D8
:10047000806489BF6BE671E082E691E0CEDF78941C
:1004800081E08093600042E0E42E0EE022E631E05D
:1004900043E065E370E088E390E0EFDDF89489B72E
:1004A0008F7B89BF8BB78F7B8BBF85B78D7F85BFD8
:1004B0000F91EF90089510926A01109269011092C5
:1004C00067010895AF92BF92CF92DF92EF92FF92B1
:1004D0000F931F93C698A0E0B0E0BC01CD012AD1D4
:1004E0005B016C0120E030E04AE753E47DD37B01FF
:1004F0008C0120E030E040E85FE321D388231CF446
:1005000081E090E020C020E03FEF4FE757E4C801D2
:10051000B70119D318169CF420E030E040E251E412
:10052000C601B50161D3A2D206C089E190E001976E
:10053000F1F76150704061157105B9F706C0C80147
:10054000B70194D2CB010197F1F7C69A1F910F9191
:10055000FF90EF90DF90CF90BF90AF9008951F92E3
:100560000F920FB60F9211248F939F9388B38F60D1
:1005700088BB88EA91E60197F1F7829BFECF88EA73
:1005800091E60197F1F780916A01882381F08091CB
:100590006701882321F015BC109260000DC0C5983A
:1005A00085B5876085BD81E08093670105C01092A5
:1005B000600081E080936A019F918F910F900FBE40
:1005C0000F901F9018951F920F920FB60F92112443
:1005D0002F933F934F935F936F937F938F939F934B
:1005E000AF93BF93EF93FF9388B38F6088BB28E8E6
:1005F00033E189E190E00197F1F721503040C9F7EC
:10060000839B05C084E690E05DDF91E006C0839B9C
:10061000FECF84EF91E056DF92E080916601813059
:10062000B9F0813030F0823019F1833009F040C0E8
:1006300030C0923059F080916501893020F48F5F8D
:100640008093650135C01092650132C081E01EC003
:10065000923059F080916401853020F48F5F80934F
:10066000640126C01092640123C09093660120C0EB
:10067000923059F080916301893020F48F5F80932C
:10068000630116C01092630113C083E0809366017A
:100690000FC0923059F080916201893020F48F5F51
:1006A0008093620105C01092620102C0109266013F
:1006B000FF91EF91BF91AF919F918F917F916F913A
:1006C0005F914F913F912F910F900FBE0F901F9010
:1006D00018950F931F93CF93DF93D9DD02E611E0B6
:1006E00084E0A0E0B0E0F801182E54D369DEC8E839
:1006F000D3E189E190E00197F1F72197D1F788ECF8
:1007000090E0E0DE80E593EC0197F1F788EC90E073
:10071000D9DE84E0DE01F801182E41D3A0DEC59AAF
:1007200088EB9BE0CFDE10926A0110926901109273
:100730006701D6CFA8E0B0E0EFE9F3E0FEC27B01AD
:100740008C01611571058105910519F482E0898399
:1007500059C083E089838EE1C82ED12CDC82CB8204
:10076000ED82FE820F831887C801B70152D0BC0109
:100770006150704077FF33C0EE27FF27E61BF70B71
:1007800020E030E040E050E081E090E0A0E0B0E028
:100790000E2E04C0880F991FAA1FBB1F0A94D2F700
:1007A0000197A109B1098E219F21A023B1230097B0
:1007B000A105B10521F021E030E040E050E004C0A7
:1007C00016950795F794E794EA95D2F72E293F29D5
:1007D000402B512B2D833E834F8358870FC06115CB
:1007E000710581F0062E04C0EE0CFF1C001F111FC6
:1007F0000A94D2F7ED82FE820F831887C61AD70AB1
:10080000DC82CB821A82CE01019650D0E8E0289695
:10081000B0C2EF92FF920F931F939B01AC01203067
:1008200080E0380781E0480780E0580780F42F3FD8
:1008300031054105510509F020F4EE24FF2487011C
:1008400019C068E0E62EF12C012D112D13C02030C7
:1008500080E0380780E0480781E0580730F490E1F5
:10086000E92EF12C012D112D05C088E1E82EF12C87
:10087000012D112D80E290E0A0E0B0E08E199F09DB
:10088000A00BB10B04C05695479537952795EA9470
:10089000D2F7F901EF59FF4F2081821B9109A1097D
:1008A000B1091F910F91FF90EF9008959F92AF9221
:1008B000BF92CF92DF92EF92FF920F931F93EE249D
:1008C000FF248701FC012481358146815781918075
:1008D0008081823010F44061A2C0843009F49BC052
:1008E000823029F420E030E040E050E005C02115DE
:1008F00031054105510519F4E0E0F0E092C0828134
:1009000093816FEF823896070CF05AC062E87FEF50
:10091000681B790B6A3171052CF020E030E040E073
:1009200050E02AC0AA24BB24650181E090E0A0E049
:10093000B0E0062E04C0880F991FAA1FBB1F0A949F
:10094000D2F70197A109B10982239323A423B523E8
:100950000097A105B10529F071E0A72EB12CC12C9B
:10096000D12C04C056954795379527956A95D2F7AF
:100970002A293B294C295D29DA01C9018F7790701A
:10098000A070B07080349105A105B10539F427FF3E
:1009900009C0205C3F4F4F4F5F4F04C0215C3F4F69
:1009A0004F4F5F4F80E090E0203060E0360760E01E
:1009B000460760E4560710F081E090E0FC0123C098
:1009C0008038910544F5FC01E158FF4FDA01C90177
:1009D0008F779070A070B07080349105A105B1053B
:1009E00039F427FF09C0205C3F4F4F4F5F4F04C0D1
:1009F000215C3F4F4F4F5F4F57FF05C056954795BE
:100A000037952795319687E05695479537952795E1
:100A10008A95D1F706C020E030E040E050E0EFEFEB
:100A2000F0E0E22EF32E942F9F77802F8078892B91
:100A30009E2F9795992797958F77082F092B9E2F93
:100A40009695812F8078892B9794992497948F7706
:100A5000182F1929C801B7011F910F91FF90EF902E
:100A6000DF90CF90BF90AF909F9008959CD088F07A
:100A70009F5790F0B92F9927B751A0F0D1F0660F8A
:100A8000771F881F991F1AF0BA95C9F712C0B130A5
:100A900081F0A3D0B1E00895A0C0672F782F8827F8
:100AA000B85F39F0B93FCCF3869577956795B395E4
:100AB000D9F73EF490958095709561957F4F8F4F53
:100AC0009F4F0895E89409C097FB3EF49095809558
:100AD000709561957F4F8F4F9F4F9923A9F0F92F04
:100AE00096E9BB279395F695879577956795B79582
:100AF000F111F8CFFAF4BB0F11F460FF1BC06F5F68
:100B00007F4F8F4F9F4F16C0882311F096E911C079
:100B1000772321F09EE8872F762F05C0662371F09A
:100B200096E8862F70E060E02AF09A95660F771FAE
:100B3000881FDAF7880F9695879597F9089507D05B
:100B400008F481E0089503D008F48FEF0895990F19
:100B50000008550FAA0BE0E8FEEF16161706E80787
:100B6000F907C0F012161306E407F50798F0621BA8
:100B7000730B840B950B39F40A2661F0232B242B7D
:100B8000252B21F408950A2609F4A140A6958FEF9C
:100B9000811D811D089557FD9058440F551F59F030
:100BA0005F3F71F04795880F97FB991F61F09F3F5A
:100BB00079F087950895121613061406551FF2CF83
:100BC0004695F1DF08C0161617061806991FF1CFD3
:100BD00086957105610508940895E894BB276627FA
:100BE0007727CB0197F908950BD078C069D028F00A
:100BF0006ED018F0952309F05AC05FC01124EECFD3
:100C0000CADFA0F3959FD1F3950F50E0551F629F67
:100C1000F001729FBB27F00DB11D639FAA27F00D55
:100C2000B11DAA1F649F6627B00DA11D661F829F7C
:100C30002227B00DA11D621F739FB00DA11D621F61
:100C4000839FA00D611D221F749F3327A00D611D7E
:100C5000231F849F600D211D822F762F6A2F112460
:100C60009F5750408AF0E1F088234AF0EE0FFF1FB3
:100C7000BB1F661F771F881F91505040A9F79E3FEA
:100C8000510570F014C0AACF5F3FECF3983EDCF33F
:100C9000869577956795B795F795E7959F5FC1F727
:100CA000FE2B880F911D9695879597F9089597F9D2
:100CB0009F6780E870E060E008959FEF80EC089502
:100CC00000240A941616170618060906089500242B
:100CD0000A9412161306140605060895092E0394A5
:100CE000000C11F4882352F0BB0F40F4BF2B11F419
:100CF00060FF04C06F5F7F4F8F4F9F4F0895AA1B07
:100D0000BB1B51E107C0AA1FBB1FA617B70710F0F6
:100D1000A61BB70B881F991F5A95A9F78095909528
:100D2000BC01CD0108952F923F924F925F926F9236
:100D30007F928F929F92AF92BF92CF92DF92EF926B
:100D4000FF920F931F93CF93DF93CDB7DEB7CA1BEC
:100D5000DB0B0FB6F894DEBF0FBECDBF09942A8817
:100D6000398848885F846E847D848C849B84AA84BF
:100D7000B984C884DF80EE80FD800C811B81AA814C
:100D8000B981CE0FD11D0FB6F894DEBF0FBECDBF17
:100D9000ED01089509D001921A94E1F708950190A8
:100DA0000BD01A94E1F70895E199FECFBFBBAEBB1B
:100DB000E09A11960DB20895E199FECFBFBBAEBB8C
:100DC0000DBA11960FB6F894E29AE19A0FBE089503
:020DD000FFCF53
:100DD20001000102020303030304040404040404E3
:100DE20004050505050505050505050505050505B2
:100DF2000506060606060606060606060606060692
:100E02000606060606060606060606060606060680
:100E12000607070707070707070707070707070761
:100E22000707070707070707070707070707070750
:100E32000707070707070707070707070707070740
:100E42000707070707070707070707070707070730
:100E52000708080808080808080808080808080811
:100E62000808080808080808080808080808080800
:100E720008080808080808080808080808080808F0
:100E820008080808080808080808080808080808E0
:100E920008080808080808080808080808080808D0
:100EA20008080808080808080808080808080808C0
:100EB20008080808080808080808080808080808B0
:100EC20008080808080808080808080808080808A0
:020ED200080016
:00000001FF
